:100000000EC013C012C011C010C00FC00EC00DC072
:100010000CC00BC00AC009C009C007C006C011242B
:100020001FBECFEDCDBF0CD02CC0EACF1F920F92D8
:100030000FB60F9211240F900FBE0F901F901895BE
:10004000CF93DF9300D0CDB7DD2780E886BD88E071
:1000500086BD8FE187BB80E681BD78942AE832E0D7
:1000600060E3C49A3A83298389819A81AC01415023
:1000700051095A834983892BB9F7C49865BF88957C
:06008000F0CFF894FFCF61
:00000001FF
